:1000000012C02CC02BC02AC029C028C027C026C0BF
:1000100025C024C023C022C021C020C01FC01EC0D4
:100020001DC01CC01BC011241FBECFE5D4E0DEBF25
:10003000CDBF10E0A0E6B0E0EAE8FFE002C0059026
:100040000D92A437B107D9F710E0A4E7B0E001C0E2
:100050001D92AE3AB107E1F757D395C7D1CFA59A14
:100060008AE18A95F1F700C0A49A8AE18A95F1F7AE
:1000700000C0A5988AE18A95F1F700C0A4988AE1AA
:100080008A95F1F700C010928B009C9905C0809171
:100090008B008F5F80938B009D9905C080918B00B2
:1000A0008F5F80938B008AE18A95F1F700C08AE127
:1000B0008A95F1F700C08AE18A95F1F700C08AE1DC
:1000C0008A95F1F700C00895A498A598AC98AD98CA
:1000D000C6DFC5DF0895A49A8AE18A95F1F700C0CA
:1000E000A59A8AE18A95F1F700C00895A4988AE15B
:1000F0008A95F1F700C0A5988AE18A95F1F700C0CA
:10010000A49A8AE18A95F1F700C0A59A8AE18A95B6
:10011000F1F700C0089598E0882314F0A49A01C074
:10012000A4982AE12A95F1F700C0A5982AE12A951A
:10013000F1F700C0A59A880F915071F7A4988AE151
:100140008A95F1F700C0A5982AE12A95F1F700C039
:1001500093B3A59A81E094FF80E00895282FA49896
:1001600098E080E0880FA5983AE13A95F1F700C051
:100170009C998160A59A3AE13A95F1F700C09150B7
:1001800089F7222311F4A49A01C0A4989AE19A95C0
:10019000F1F700C0A5983AE13A95F1F700C0A59AA9
:1001A0009AE19A95F1F700C0A4980895CF93DF9350
:1001B000C82F91DF8EEEAFDF8C2FADDF50DF8BDFEE
:1001C0008FEEA9DF80E0CADFD82F81E0C7DFC82F1C
:1001D00046DF3D2F20E0C9018C0F911DDF91CF91AB
:1001E00008958AEAE3DF90939500809394008CEA67
:1001F000DDDF90939D0080939C008EEAD7DF909383
:10020000AD008093AC0080EBD1DF9093A100809390
:10021000A00082EBCBDF90939B0080939A0084EB4D
:10022000C5DF909399008093980086EBBFDF909391
:1002300097008093960088EBB9DF909391008093AC
:1002400090008AEBB3DF90939300809392008CEB45
:10025000ADDF9093A3008093A2008EEBA7DF909375
:100260009F0080939E00089536DF8EEE54DF84EF6A
:1002700052DF8EE250DFF3DE8FE097E20197F1F775
:1002800000C0000086EF92DFA0E0B0E080937B002A
:1002900090937C00A0937D00B0937E0008951BDFB7
:1002A0008EEE39DF84EF37DF84EF35DFD8DE8FE184
:1002B0009BEC0197F1F700C000000DDF8EEE2BDF05
:1002C00086EF29DFCCDE07DF8FEE25DF80E046DF1B
:1002D00090E0A0E0B0E08093A8009093A900A093E4
:1002E000AA00B093AB0080E039DF90E0A0E0B0E07E
:1002F0008093A4009093A500A093A600B093A700BC
:1003000081E02CDF90E0A0E0B0E080938C0090933F
:100310008D00A0938E00B0938F00A1DE4091A800C5
:100320005091A9006091AA007091AB00BA015527C5
:1003300044278091A4009091A500A091A600B091BF
:10034000A700BA2FA92F982F8827840F951FA61FC3
:10035000B71F40918C0050918D0060918E0070917C
:100360008F00840F951FA61FB71F689414F8B695C9
:10037000A795979587951694D1F7809377009093DA
:100380007800A0937900B0937A0008954F925F921D
:100390006F927F928F929F92AF92BF92CF92DF9295
:1003A000EF92FF920F931F93CF93DF93CDB7DEB7FA
:1003B0002C970FB6F894DEBF0FBECDBF4C018B015A
:1003C00053DFC0907B00D0907C00E0907D00F090E7
:1003D0007E0065DF209177003091780040917900B0
:1003E00050917A002D833E834F83588780919800E7
:1003F00090919900A0E0B0E0A7019601281B390B6D
:100400004A0B5B0BCA01B90120919A0030919B0005
:1004100040E050E05CD56B017C010B2EBFE0F59411
:10042000E794D794C794BA95D1F7B02D6091A20004
:100430007091A300CB01AA2797FDA095BA2FBC010C
:10044000CD01052E5BE0660F771F881F991F5A9517
:10045000D1F7502D20919E0030919F00442737FD09
:100460004095542F2C0D3D1D4E1D5F1D71D5C20EA4
:10047000D31EE41EF51ED701C6010896A11DB11DAD
:10048000689413F8B595A795979587951694D1F725
:10049000F40180839183A283B38320E630EF4FEF92
:1004A0005FEFC20ED31EE41EF51EC701B601A70101
:1004B00096010DD5DC01CB019C01AD01012E1CE0A4
:1004C00055954795379527951A95D1F7102D29837E
:1004D0003A834B835C836091AC007091AD008827B8
:1004E00077FD8095982FA7019601F1D44B015C010F
:1004F000072E7DE0B594A794979487947A95D1F7C9
:10050000702D2091960030919700442737FD40953B
:10051000542F69817A818B819C81D9D4DC01CB01F4
:10052000CD01BB2797FDB095AB2F880D991DAA1D56
:10053000BB1D0296A11DB11DB595A79597958795F1
:10054000B595A79597958795BC01CD0160507048EA
:100550008F4F9F4F2091A0003091A10040E050E0CC
:10056000B6D4DC01CB019C01AD01012E1FE05695F4
:100570004795379527951A95D1F7102D29873A87F2
:100580004B875C874090940050909500662457FC00
:100590006094762C440C551C661C771C440C551C2E
:1005A000661C771C6091900070919100882777FD00
:1005B0008095982F29813A814B815C8188D44B01A9
:1005C0005C01072E7BE0B594A794979487947A9565
:1005D000D1F7702D60919C0070919D00882777FD68
:1005E0008095982FA701960172D4DC01CB01072ECC
:1005F0007BE0B595A795979587957A95D1F7702D5E
:10060000880E991EAA1EBB1E840C951CA61CB71C26
:10061000880C991CAA1CBB1C6D817E818F819885DA
:10062000681979098A099B092AE638E140E050E017
:100630004ED4992364F0660F771F881F991F298570
:100640003A854B855C8562D469017A010BC02985A6
:100650003A854B855C855AD469017A01CC0CDD1C46
:10066000EE1CFF1C5527F7FC5A954F2D3E2D2D2DC6
:10067000CA01B9012CD42EED3BE040E050E027D474
:100680004C01BB2497FCB094AB2CC701B60123E40A
:1006900033EE4FEF5FEF1BD4DC01CB01CD01BB2765
:1006A00097FDB095AB2F880D991DAA1DBB1D8153D9
:1006B000914FAF4FBF4F689413F8B595A795979595
:1006C00087951694D1F7C80ED91EEA1EFB1ED801D5
:1006D000CD92DD92ED92FC9213972C960FB6F89482
:1006E000DEBF0FBECDBFDF91CF911F910F91FF9065
:1006F000EF90DF90CF90BF90AF909F908F907F90C2
:100700006F905F904F900895CF93DF9300D0CDB757
:10071000DEB745D2D9DC65DD81E005D28FE99FE007
:100720000197F1F700C000000F2EF7E82F2EF0E040
:100730003F2EF02D0F2EF8EE4F2EF3E05F2EF0E05F
:100740006F2EF0E07F2EF02DC10163E870E01EDE19
:10075000C0908300D0908400E0908500F0908600E7
:10076000C701B601A3019201F3D34901A8E1BCEF8F
:100770002A9FC0012B9F900D3A9F900D11245C0180
:10078000AC0CBD1CC701B60116D32FE632E545E01F
:1007900053E476D2DDD2DC01CB019A838983C09009
:1007A0008700D0908800E0908900F0908A00C7010F
:1007B000B6012AE030E040E050E0CAD3122F822F89
:1007C000932F880F991F9C01220F331F220F331F75
:1007D000820F931F909581959F4FC80ED91EE09070
:1007E0007400F0907500EA14FB0434F4C5018E190E
:1007F0009F098F30910564F0AE14BF0444F4C70123
:100800008A199B098F3091051CF0750101C0750193
:10081000F0927500E092740080E885D1812F30D08D
:100820008CE29FD18C2D29D080E690E0EAD187E838
:100830007AD189819A815FD083E690E0E2D15FD15D
:100840008093760080EC6FD18091760019D08AE693
:1008500090E0D7D187EC67D1C4014DD0C7014BD010
:100860008FE690E0CED18FEF93EDA0E381509040E2
:10087000A040E1F700C0000067CF805D72D108950D
:10088000CF93C82F8A3048F080E08F5FCA50CA30BB
:10089000E0F7882321F0805D03C080E301C080E39E
:1008A00060D18C2F805D5DD1CF910895CF93C82FFB
:1008B000843648F080E08F5FC456C436E0F7882362
:1008C00021F0805D03C080E301C080E34AD1CA30DB
:1008D00048F080E08F5FCA50CA30E0F7882321F0EB
:1008E000805D03C080E301C080E33BD18C2F805D3D
:1008F00038D1CF910895CF93DF93EC0184369105E1
:1009000058F080E08F5FC456D040C436D105D0F790
:10091000882321F0805D03C080E301C080E321D102
:10092000CA30D10550F080E08F5F2A97CA30D105D8
:10093000D8F7882321F0805D03C080E301C080E305
:1009400010D18C2F805D0DD1DF91CF910895CF9381
:10095000DF93EC0183E0C83ED80760F080E08F5F52
:10096000C85ED34093E0C83ED907C8F7882321F07A
:10097000805D03C080E301C080E3F3D0C436D105BD
:1009800058F080E08F5FC456D040C436D105D0F710
:10099000882321F0805D03C080E301C080E3E1D0C3
:1009A000CA30D10550F080E08F5F2A97CA30D10558
:1009B000D8F7882321F0805D03C080E301C080E385
:1009C000D0D08C2F805DCDD0DF91CF910895FF9254
:1009D0000F931F93CF93DF9300D000D00F92CDB72A
:1009E000DEB7482FFE01319685E0DF011D928A9522
:1009F000E9F7A39AAB9A8FEF90E7A2E0815090407D
:100A0000A040E1F700C00000AB98AFE9BCE8119747
:100A1000F1F700C00000AB9AB2E0BA95F1F700C060
:100A2000A39888E68A95F1F79B9954C095ED9A951D
:100A3000F1F700009B9B50C0A5EDAA95F1F70000CF
:100A4000FE0131968E010A5F1F4FA7E0B0E0FF2440
:100A500061E070E01BC09B9BFECF80E58A95F1F7BB
:100A60009B9B08C0CB01022E02C0880F991F0A94DD
:100A7000E2F7582B9B99FECF215030409FEF2F3F3C
:100A8000390749F75193E017F10719F09D015F2DE0
:100A9000E2CFA39AAB9A8FEF90E7A2E0815090400B
:100AA000A040E1F700C0000099818B816A8170E06D
:100AB000690F711D680F711D2C81620F711D2D81D1
:100AC00030E06217730751F4442359F0413041F08C
:100AD0008FEF07C08FEF05C08FEF03C08FEF01C00E
:100AE000892F0F900F900F900F900F90DF91CF9163
:100AF0001F910F91FF90089580E069DF089581E0D4
:100B000066DF08959AE69A95F1F700C0909892B33F
:100B1000807F9F70892B82BB929A85E08A95F1F73E
:100B20000000929808959AE69A95F1F700C090987F
:100B300092B3282F207F9F70922B92BB929A95E0C0
:100B40009A95F1F70000929892B38295807F9F70FA
:100B5000892B82BB929A85E08A95F1F700009298E2
:100B600008959AE69A95F1F700C0909A92B3282FCB
:100B7000207F9F70922B92BB929A95E09A95F1F705
:100B80000000929892B38295807F9F70892B82BBE0
:100B9000929A85E08A95F1F700009298089581B3C2
:100BA000806F81BB889A899A8A9A8FEF99EFA0E02B
:100BB00081509040A040E1F700C0000080E3A2DF38
:100BC000AFE1BEE41197F1F700C0000080E39ADFC7
:100BD0008FE99FE00197F1F700C0000080E392DF0A
:100BE00088E290DF88E29FDF8CE09DDF81E09BDF81
:100BF000AFE9BFE01197F1F700C0000086E093DF96
:100C00000895CF93DF93EC018881882329F0219602
:100C1000A8DF89918823E1F7DF91CF910895CF93E1
:100C2000DF93EC018881882341F02196FE01319702
:100C3000849197DF89918823C9F7DF91CF91089537
:100C40000F931F93CF93DF938C01862F90E08770D3
:100C50009070880F991F880F991F880F991F8064C3
:100C600062DFE8012896F80184910F5F1F4F79DF5A
:100C70000C171D07C1F7DF91CF911F910F910895B8
:100C80000CD0EBC0E3D040F0DAD030F021F45F3F7D
:100C900019F0CCC0511115C1CFC0F0D098F39923F1
:100CA000C9F35523B1F3951B550BBB27AA27621730
:100CB0007307840738F09F5F5F4F220F331F441F75
:100CC000AA1FA9F333D00E2E3AF0E0E830D09150AD
:100CD0005040E695001CCAF729D0FE2F27D0660F9A
:100CE000771F881FBB1F261737074807AB07B0E8D9
:100CF00009F0BB0B802DBF01FF2793585F4F2AF0EF
:100D00009E3F510568F092C0DCC05F3FECF3983E17
:100D1000DCF3869577956795B795F7959F5FC9F74B
:100D2000880F911D9695879597F90895E1E0660FD4
:100D3000771F881FBB1F621773078407BA0720F04D
:100D4000621B730B840BBA0BEE1F88F7E0950895B6
:100D500004D06894B111B5C0089598D088F09F5719
:100D600090F0B92F9927B751A0F0D1F0660F771FF7
:100D7000881F991F1AF0BA95C9F712C0B13081F0D7
:100D80009FD0B1E008959CC0672F782F8827B85F67
:100D900039F0B93FCCF3869577956795B395D9F738
:100DA0003EF490958095709561957F4F8F4F9F4F42
:100DB0000895E89409C097FB3EF49095809570954E
:100DC00061957F4F8F4F9F4F9923A9F0F92F96E997
:100DD000BB279395F695879577956795B795F1110C
:100DE000F8CFFAF4BB0F11F460FF1BC06F5F7F4FA9
:100DF0008F4F9F4F16C0882311F096E911C07723BB
:100E000021F09EE8872F762F05C0662371F096E8C3
:100E1000862F70E060E02AF09A95660F771F881F92
:100E2000DAF7880F9695879597F9089597F99F6750
:100E300080E870E060E008959FEF80EC0895002462
:100E40000A941616170618060906089500240A942F
:100E500012161306140605060895092E0394000CB5
:100E600011F4882352F0BB0F40F4BF2B11F460FF44
:100E700004C06F5F7F4F8F4F9F4F089557FD90586D
:100E8000440F551F59F05F3F71F04795880F97FB4E
:100E9000991F61F09F3F79F0879508951216130608
:100EA0001406551FF2CF4695F1DF08C01616170637
:100EB0001806991FF1CF869571056105089408956C
:100EC000E894BB2766277727CB0197F90895629F9F
:100ED000D001739FF001829FE00DF11D649FE00D32
:100EE000F11D929FF00D839FF00D749FF00D659F93
:100EF000F00D9927729FB00DE11DF91F639FB00D92
:100F0000E11DF91FBD01CF0111240895A1E21A2EA0
:100F1000AA1BBB1BFD010DC0AA1FBB1FEE1FFF1F9D
:100F2000A217B307E407F50720F0A21BB30BE40BED
:100F3000F50B661F771F881F991F1A9469F7609534
:100F40007095809590959B01AC01BD01CF010895EE
:100F500097FB092E05260ED057FD04D0D7DF0AD007
:100F6000001C38F450954095309521953F4F4F4FD8
:100F70005F4F0895F6F790958095709561957F4F36
:0A0F80008F4F9F4F0895F894FFCFA4
:100F8A00204300206D6D204867002025526800200C
:040F9A0050610000A2
:00000001FF
